:020000040800F2
:1000000000200020E50E0008250E0008290E00083B
:1000100000000000000000000000000000000000E0
:100020000000000000000000000000002D0E00088D
:100030000000000000000000310E0008350E00082E
:10004000350F0008350F0008350F0008350F000880
:10005000350F0008350F0008350F0008350F000870
:1000600000000000350F0008350F0008350F0008AC
:10007000350F0008350F000800000000350F00089C
:1000800000000000350F0008000000000000000024
:100090003D0E000800000000350F0008350F000875
:1000A000350F0008350F0008350F00084D0E000809
:1000B000350F0008350F00080000000000000000A8
:1000C00010B5064C2378002B07D1054B002B02D02E
:1000D000044800E000BF0123237010BD040000208D
:1000E0000000000008270008044B10B5002B03D0C7
:1000F0000349044800E000BF10BDC04600000000F6
:100100000800002008270008002243088B4274D30F
:1001100003098B425FD3030A8B4244D3030B8B4208
:1001200028D3030C8B420DD3FF22090212BA030C11
:100130008B4202D31212090265D0030B8B4219D3F2
:1001400000E0090AC30B8B4201D3CB03C01A524112
:10015000830B8B4201D38B03C01A5241430B8B425A
:1001600001D34B03C01A5241030B8B4201D30B0343
:10017000C01A5241C30A8B4201D3CB02C01A52416A
:10018000830A8B4201D38B02C01A5241430A8B422D
:1001900001D34B02C01A5241030A8B4201D30B0216
:1001A000C01A5241CDD2C3098B4201D3CB01C01A30
:1001B000524183098B4201D38B01C01A524143093A
:1001C0008B4201D34B01C01A524103098B4201D328
:1001D0000B01C01A5241C3088B4201D3CB00C01A95
:1001E000524183088B4201D38B00C01A524143080D
:1001F0008B4201D34B00C01A5241411A00D2014632
:10020000524110467047FFE701B5002000F006F8A4
:1002100002BDC0460029F7D076E770477047C04658
:10022000002B11D1002A0FD1002900D1002802D0C3
:100230000021C943081C07B4024802A140180290DB
:1002400003BDC046D9FFFFFF03B4684601B502985D
:1002500000F006F8019B9E4602B00CBC7047C046F9
:10026000F0B54F464646D646C0B5040082B00D00F4
:10027000914698468B422FD82CD04146484600F0F4
:10028000B1F829000600200000F0ACF8331A9C46B3
:10029000203B9A4600D576E04B46524693401F00DD
:1002A0004B46624693401E00AF4228D825D05346A5
:1002B000A41BBD41002B00DA7BE00022002300924A
:1002C00001930123524693400193012362469340D8
:1002D000009318E08242D0D90022002300920193BB
:1002E0000A9B002B01D01C605D600098019902B050
:1002F0001CBC90469946A246F0BDA342D7D9002225
:100300000023009201936346002BE9D0FB07984637
:10031000414672080A437B0866460EE0AB4201D1B3
:10032000A2420CD8A41A9D41012024196D4100213C
:10033000013E24184D41002E06D0AB42EED9013EBD
:1003400024196D41002EF8D10098019953460019E7
:100350006941002B23DB2B005246D3402A00644620
:10036000E2401C0053461500002B2DDB26005746AB
:10037000BE40330026006746BE403200801A9941D5
:1003800000900191ACE7624620239B1A4A46DA406E
:100390006146130042468A4017001F4380E76246C9
:1003A00020239B1A2A0066469A402300F3401343F9
:1003B000D4E76246202300219B1A0022009101927B
:1003C0000122DA40019280E72023624626009B1A30
:1003D000DE402F00B0466646B74046463B003343FA
:1003E000C8E7C04610B5002903D100F007F8203057
:1003F00002E0081C00F002F810BDC0461C210123D9
:100400001B04984201D3000C10391B0A984201D3F7
:10041000000A08391B09984201D30009043902A2D5
:10042000105C40187047C04604030202010101013C
:100430000000000000000000F0B54F464646D646DA
:10044000164BC0B599461E68154B00259846154FAA
:1004500007E0E41A0134E4B27C5501353619802DE9
:1004600015D0EBB29A464346A8B25B1903215C7BD8
:10047000FFF7D0FE89B2E4B253460029E9D1023B2E
:10048000E418E4B27C5501353619802DE9D14B468C
:100490001E601CBC90469946A246F0BDA4010020F7
:1004A000AC01002034000020F8B580231B05C418DF
:1004B000104B9C421AD9104B0025C7180F4E03E071
:1004C00004340135A74213D0AB00F25CF31859781D
:1004D0000220090211439A7812041143DA781206B5
:1004E0000A43210000F098FE0028E9D00020F8BD62
:1004F0000130FCE7FF3F00088000000834000020C6
:1005000030B59BB02C2200210FA802F0F4F8142281
:10051000002101A802F0EFF81C22002106A802F039
:10052000EAF81249124A0B6800241A4080231B0182
:1005300013430B60802301255B020DA80E930D95DC
:10054000169401F02DF80F230021019301A80D3B13
:10055000029303940494059401F0BEFA06A806954C
:10056000089401F0A1FB1BB030BDC04600700040F4
:10057000FFE7FFFFA0239C2210B5134CE35CDBB226
:10058000181D0533DBB2C0B2A35400281AD00022D4
:100590000023A1189D3109780132CB18D1B2DBB20A
:1005A0008142F6D320189D30037001229B23202125
:1005B0000648E25400F0A2FF9D23E35C044ADBB24C
:1005C000936210BD0023EDE7AC0100200004005051
:1005D00000380140F0B54E464546DE465746E0B588
:1005E000CE4CCF4D23792E78DBB283B0B34206D008
:1005F00003B03CBC90469946A246AB46F0BDE278BB
:10060000A779D2B2FFB29046012F2BD0022F1FD074
:10061000032F00D07BE10022C24B91461B78012BB7
:1006200000D11BE19D232A22E25442460133E654C5
:100630000133E25403220133E25401336132E254C4
:100640004A460133E7540133E254FFF793FFCFE703
:10065000B44B9A461B789946012B00D1EAE000235F
:100660009946DFE7E279D2B2012A52D00021AD4BA0
:100670001970022A01D1FE23A3710022A3799146A9
:10068000DBB2052BCED0092B23D0FE2BCAD19D2265
:100690002A21A15441460132A6540132A154042119
:1006A0000132A1540132A3545C3B8B3AE254AB7843
:1006B0008D32E978A05CA3542300A3335878597095
:1006C00069780129C1D0A15C0021A1545A785970E0
:1006D000BBE7944B1B78012BA4D10020E279217A4F
:1006E000814609021143627A12041143A27A12066A
:1006F0000A438D4909688A4294D10422290001A83D
:100700006B7001F0EFFF894B019A1A600123994643
:1007100088E784492A200A709D216054013163547E
:1007200041469F23E15418210133E1540133E2543F
:100730000133E2540133E25C1622E2542300002725
:10074000A3335A785F70A523E25C0222E2542300AF
:10075000A5335978A721FF2688465A70EB78AA78E6
:100760001B0213433200615C41461A406254A722C7
:100770009146A1444A4652784A461B0A5370A9231F
:10078000E25CE7542300A9335A78012252425A709E
:10079000AB23E25C80225242E2542300AB335A780E
:1007A0005F7000F003FC3200AD230240E15CE254D4
:1007B0002300020AAD33324059785A70020C32409D
:1007C0009978000E9A70DA78D87000F0F5FB320054
:1007D000B1230240E15CE2542300020AB13332400B
:1007E00059785A70020C32409978000E9A70DA7873
:1007F000D87000F0E7FB3200B5230240E15CE25420
:100800002300020AB533324059785A70020C164060
:10081000000E9A789E70DA78D8706B78012B00D130
:1008200013E74346E35C4346E7544B465B784B464D
:100830005F700AE7E379DBB29A1ED2B2FC2A00D9D4
:100840000DE70422290001A82B7001F04BFF374B64
:10085000019A1A60002352461370E3E6227AE37984
:1008600012029B189BB2AB701B0AEB704B46042222
:10087000290001A86B7001F035FF019A2B4B2C4821
:100880001A604A46284B2B491A60FF222A4B12064F
:100890001A604B460360294B4360C0235B008360B2
:1008A00000F0D8FC43425841A379C0B2DBB2052B1B
:1008B00032D11C4B1B789946012B2BD1E379227A3C
:1008C00012021A43637A1B041A43A37A1B061343CA
:1008D0001B4A13609346184A92461268934211D0FD
:1008E000FFF7AAFD53461A685B461868824208D093
:1008F000FFF7DAFD013843424341DBB299465B46DC
:100900001A68A37953461A60A379DBB2BBE63B00B1
:100910000020CCE7814685E68146B4E6AC010020A4
:10092000D8000020DC000020A401002000000808FE
:10093000200000202C000020E000002000400008E3
:10094000A0010020F0B5DE46454657464E46E0B5CC
:100950008BB000AF00F008FBFFF7D2FD00F0E6FB24
:10096000142314220021F81801F0C5FE8022884BC0
:100970000126D96A87481143D962D96A80250A407D
:100980003A603A680222D96A00241143D962D96ACE
:100990006D010A407A607A68DA6A7F493243DA6226
:1009A000DB6A00223340BB60BB6800F0A7FD142364
:1009B0007848F9187D61BC61FC6100F0ABFC142340
:1009C000754AF91873487A61BE61FC613C6200F0B7
:1009D000A1FC7248724B0B3603609623DB01436027
:1009E0008460C460046146618461C46104624462DD
:1009F00001F020FE14231022F818002101F07BFEE4
:100A00000C2000210822381801F075FE654A664B5B
:100A10001000136078235360644B9460D3601461BA
:100A2000546101F047FA14235E48F9187D6101F022
:100A3000A1FA0C2039185B48FC603C6101F0D8FB3E
:100A400014231022F818002101F055FE0C2000217B
:100A50000822381801F04FFE554A564B100013601B
:100A6000FA23DB00D360566094601461546101F096
:100A700021FA14234E48F9187D6101F07BFA0C200D
:100A800039184B48FC603C6101F0B2FB2900414839
:100A900000F02EFD484B9846002869D00C23474DA6
:100AA00004222C68F918FC60023C4046E4B201F0D4
:100AB00019FEFC2C4CD81E23414A13700022414BD6
:100AC0001A7042465278012A01D003221A70354822
:100AD00001F030FA364801F007FA4021304B9A25F0
:100AE0001A6A99460A431A621A6820310A431A6040
:100AF000354A364E9346364A9246735D002B22D1D4
:100B00002F4B1C78E4B2002CF7D143465B78012BC5
:100B1000F3D100F039FB4B4622481C621C6001F007
:100B200019FA234801F0F2F972B65A46294B1B68AC
:100B3000136052461360284A126882F30888984767
:100B4000735D002BDCD0FFF745FD00237355D7E71D
:100B50004246FE231370002353709370D3701433F6
:100B6000F8180422414601F0BDFD7B692B60A2E725
:100B70004246FE231370142350709070D07041468B
:100B80000422F81801F0AEFD0C4B7A691A6085E773
:100B9000001002400004005020400000200100200E
:100BA00000380140E002002000080140102700004A
:100BB000E400002000140140D800002000000808D4
:100BC000DF020020DC000020D4000020AC01002067
:100BD000A801002004400008004000089A2230B517
:100BE000304B596A304B9A5CD2B2002A16D12F484A
:100BF00000680469E40703D599241D5D012D1AD00E
:100C000099241A5DC9B2D2B2002A08D099229C5CFC
:100C1000012C12D000234362023B036130BD2A291C
:100C2000F4D102256D42426205611A7098329954DE
:100C3000973A1A55F2E71A55E2E71C780134E4B204
:100C40001C701C788C2C01D900249C5498241A7890
:100C50009A1891701A5D5218D2B21A551A78032A4E
:100C600015D01C785A789442D4D198241A5D521A1F
:100C7000D2B21A551A5D8A42CCD199215A5CD2B2AD
:100C8000012AC7D102341A5500225A54C2E70A1D5C
:100C9000D2B25A705A788C2AE3D9992200249C54F3
:100CA000DFE7C04600380140AC010020E40000202E
:100CB0009B229C2110B50B4B985C595C88420BD24F
:100CC000995C094859189D310978C9B28162995CCB
:100CD0000131C9B2995410BD00222021034800F00F
:100CE0000DFCF8E7AC010020003801400004005082
:100CF000154B10B5984200D010BD144A144C13780F
:100D00000133DBB213702378012B02D01378DB0799
:100D100012D480210122C9010E4800F0EFFB237894
:100D2000002B05D10C4A1378013BDBB21370E3E7CB
:100D30001E22094B1A70DFE780210022C9010548F5
:100D400000F0DCFBEBE7C046E002002030000020B2
:100D5000DC00002000040050DF0200200121054BD0
:100D60005A6B0A435A638022996B52050A439A636D
:100D70007047C0460010024003680D4A10B5934208
:100D800008D00C4A934204D120210B4A536B0B43E9
:100D9000536310BD0421084A1420536B0B43536363
:100DA0000021002200F014F9142000F03DF9F0E7D2
:100DB00000080140001401400010024010B504007A
:100DC00086B01422002101A801F095FC124B226884
:100DD0009A4201D006B010BD8022104BD201596B4F
:100DE0000F480A435A630222D96A1143D962DB6A67
:100DF00001A913400093009BC0230193BD3B0292C5
:100E0000049300F087FA002200211B2000F0E0F894
:100E10001B2000F009F9DDE7003801400010024016
:100E2000000400507047C046FEE7C0467047C04609
:100E30007047C04610B500F0ABF810BD10B50248C1
:100E400001F048F910BDC046E002002020230D4A01
:100E500070B5D1690B4202D0126813420ED1402501
:100E6000084CE3691D4202D023681D4200D170BDC9
:100E7000FFF71EFF236A1D432562F8E7FFF7AEFE6A
:100E8000EDE7C046003801408022104B520019683F
:100E90000A431A60DA680E490A40DA601A680D4996
:100EA0000A4001211A609A688A439A601A680A49BE
:100EB0000A401A60DA6809490A40DA6000221A61B9
:100EC0008022074B12059A607047C046001002400E
:100ED0000C40FF88F6FFF6FEFFFFFBFFFFFF02FF5F
:100EE00000ED00E00D488546002103E00C4B5B5807
:100EF000435004310B480C4B42189A42F6D30B4A2C
:100F000002E0002313600432094B9A42F9D3FFF741
:100F1000BBFF01F0C3FBFFF715FDFEE7002000203B
:100F2000B02700080000002004000020040000207A
:100F300038030020FEE70000FA210A4B10B58900B3
:100F400004001868FFF7E0F800F078F801230028A3
:100F500005D100222100013800F03AF800231800E2
:100F600010BDC046000000204021084A10B513689B
:100F700000200B431360FFF7DFFF041E02D00124A3
:100F8000200010BDFFF7EAFEFAE7C046002002404D
:100F9000024A1368013313607047C0461C030020E7
:100FA000014B18687047C0461C030020014B1868AD
:100FB0007047C0465000F81F014B18687047C04684
:100FC0005400F81F014B18687047C0466400F81FB2
:100FD000FF22032330B51400C5B22B40DB009C4038
:100FE00089010A40E4439A4000280BDB0C4B80083F
:100FF0009C46C023800060449B00C1580C402243A3
:10100000C25030BD0F2307492B408C46083B9B083C
:101010009B006344D9690C402243DA61F1E7C04682
:1010200000E100E000ED00E01F2318401E3B83407C
:10103000014A13607047C04600E100E00A4A431EBF
:10104000012093420ED8C021084A09485360036A20
:1010500009061B021B0A0B43036200230020936056
:10106000073313607047C046FFFFFF0010E000E049
:1010700000ED00E080222B4B5200996910B500234F
:10108000114205D0022028494B6903434B611300EC
:10109000244A916980229200114205D001242248FD
:1010A00013434169214341611E4A91698022D20064
:1010B000114205D008241C48134341692143416172
:1010C000184A916980221201114205D00424164861
:1010D0001343416921434161124A9169802292017F
:1010E000114205D010241048134341692143416146
:1010F0000C4A9269920305D520210B480B434269A3
:101100000A434261074A916980225202114205D086
:10111000402405481343416921434161014A9361D9
:1011200010BDC04600200240200300200122114BC8
:1011300059680A420CD0EFF3108172B60E48D8609D
:101140000E48D86081F310885B6801201A4210D1E4
:10115000084B00205A6892070BD5EFF3108272B645
:10116000074919610749196182F310885868800797
:10117000C00F704700200240EFCDAB890504030289
:10118000BFAE9D8C161514130221054B00205A6822
:101190000A435A605A6801390A435A607047C04688
:1011A00000200240F8B50500FFF7FAFE194C0700D1
:1011B000012601E06B1C11D1A3691E42FAD1022362
:1011C000A269134213D1134B9A69D20502D49A69CA
:1011D00092050ED5FFF74EFF0120F8BD002D04D07B
:1011E000FFF7DEFEC01BA842E6D90320F5E7A361A6
:1011F000E9E79A695205EDD49A691205EAD49A6929
:101200009204E7D49A699203E4D49B690020DB033B
:10121000E0D4E2E70020024070B50C4C0D00237CC6
:101220001600012B0FD0012309482374FFF7BAFFE2
:10123000002802D00023237470BD60612E60044832
:10124000FFF7B0FFF6E70220F6E7C04620030020D4
:1012500050C30000F8B557464E46DE464546E0B559
:10126000284F06003B7C8A46012B47D001232648A5
:101270003B74FFF797FF8146031E36D15246013B70
:101280001360B3687568DB015B199D422DD20023A2
:101290001E4C984607E07268B3689446DB018035BF
:1012A0006344AB4221D943467B61802362689B0043
:1012B00013430822636063689346134363602A0004
:1012C0007F239A43130042460F481A60FFF76AFFD4
:1012D0005A4663689343636063680D4A13406360D2
:1012E0000028D8D0534681461D6000233B744846F1
:1012F0003CBC90469946A246AB46F8BD02239946AF
:10130000F5E7C0462003002050C300000020024043
:10131000FFFDFFFFF0B5DE4657464E464546E0B5B9
:101320000B6883B09C46002B00D184E001239A46D1
:10133000684B0022984663460191009354469440BE
:10134000009D254073D0019B10275B681900B943AD
:101350008946022900D175E051008C46032166467A
:10136000B14001267642B346D9444E46C943012EC8
:1013700000D887E0046867460C40A14603241C405F
:10138000BC404F463C4367460460C4680C4001992A
:101390008968B9402143C160802149050B4246D08C
:1013A000564603274C4C1740616B314361634B4CED
:1013B000BE00A4460F27910889006144B740B44697
:1013C000A0268C68F605BC43B04215D0444EB0420E
:1013D00000D175E0434EB1460226484509D0424E41
:1013E000B04200D171E0414EB1460526484500D0DB
:1013F00006266746BE4034438C604146EC4309688C
:10140000DE035BD421404646316071689E0353D4AD
:10141000214046467160B168DE024BD42140464609
:10142000B160F1689B0243D421404346D960009BE0
:101430000132D34082D103B03CBC90469946A246CB
:10144000AB46F0BDD108890041180E6AB1460726A7
:1014500037001740BE000F27B740BB46B4464F4683
:101460005E46B743019EB94637696646B740BC46FB
:101470004F46664637430F6251008C46032166464D
:10148000B140C9438768019E0F40BB46F768664676
:10149000B740B9465F464E463743876046683700D7
:1014A0005646A7431C09344094403C43446061E7DE
:1014B0002943BAE72943B2E72943AAE72943A2E728
:1014C00056466746BE40344396E703266746BE400D
:1014D000344391E700040140001002400000014045
:1014E0000004005000080050000C0050001C005088
:1014F00000690840411E8841C0B27047002A01D1EE
:10150000816270478161FCE70C23204A10B5D168E5
:101510000B40082B2BD00C2B12D0042B07D0802093
:10152000536800021B045B0F0133984010BD106824
:10153000174BC006C0171840164B9C466044F5E791
:101540008B0215481B0FC05C0902D368890F01315B
:10155000DB030ED413684201121ADB060ED5930189
:101560009B1ADB0018180002FEF7CEFDDEE70B48E1
:10157000DCE70A4B5843FEF7C7FDD7E793019B1AF8
:10158000DB0018188002FEF7BFFDCFE70010024015
:1015900000E548FF0024F40038270008001BB700CE
:1015A000F0B5D6464F464646C0B5040082B0002886
:1015B00000D11FE10C258026C64B7602DA68154063
:1015C000DA6803681640DA0733D5082D00D108E140
:1015D0000C2D00D102E1802061684002814200D1DF
:1015E0005FE1A022D202914200D131E2B94FBA4B61
:1015F0003A681A403A603B68B84A03400193019B3D
:101600003B6813403B60002900D04EE1FFF7C8FC67
:1016100080239B028146984606E0FFF7C1FC4B46BB
:10162000C01A642800D998E142463B681342F4D1BD
:1016300023689A0700D5ABE0DA062AD5002D00D141
:10164000DFE0A369A34E002B00D1B2E18023326812
:101650005B0013433360FFF7A3FC80278046BF0085
:1016600006E0FFF79DFC4346C01A022800D974E14A
:1016700033683B42F5D07368994A1340226A13439A
:1016800073607268E36912021B06120A13437360E7
:1016900023681A0719D563698E4E002B00D173E1B8
:1016A0000122336D13433365FFF77AFC02230700F1
:1016B000984605E0FFF774FCC01B022800D94CE1F6
:1016C0004246336D1A42F5D023685B0741D580232B
:1016D0000020804A5B05916B8246194204D1916BD0
:1016E0000B43936301239A4680277E4E7F00336825
:1016F0003B4200D121E18022A3685200934200D1F5
:10170000B0E1002B00D1FDE0A021C9008B4200D147
:10171000CAE1704B74491A6D0A401A651A6D734913
:101720000A401A65FFF73CFC8026714B8146694FE1
:10173000B600984606E0FFF733FC4B46C01A40451A
:1017400000D90AE13B6D3342F5D05346012B00D15D
:1017500078E1636A002B19D00C2D00D187E1022BB0
:1017600000D13CE15B4C634A236880251340236031
:10177000FFF716FCAD04060005E0FFF711FC801B27
:10178000022800D9E9E023682B42F6D1002032E09C
:10179000E368042D61D00C2D5DD04E4E002B00D19E
:1017A000DDE00921326804278A4313433360FFF7E1
:1017B000F7FB804606E0FFF7F3FB4346C01A02281A
:1017C00000D9CAE033681F42F5D0726823694A49DC
:1017D0001B020A401343736023682DE7002E00D1DB
:1017E000F9E63C4A1268920300D422E76268002AB4
:1017F00000D01EE7012002B01CBC90469946A246CC
:10180000F0BD344B1B689B0502D5A369002BF1D0BA
:10181000304A33485168236A014019435160506887
:10182000E1690002000A090601435160D168802283
:101830005B0B013312029A4013000A062F49120F64
:101840008A5C0020D3402E4A1360FFF775FB002806
:10185000D1D123681DE7002E9FD11E4A126852077E
:1018600001D5002BC6D01B4E226971682248120296
:1018700001400A430921726032688A43134333608E
:10188000FFF742FEF3681D4A1B061B0FD35CD840CE
:101890001B4B18600020FFF74FFB0028ABD12368DB
:1018A000CAE60C4A13680B431360FFF779FB8027E5
:1018B000084B81469846BF0205E0FFF771FB4B4697
:1018C000C01A642849D843461B683B42F5D02368B8
:1018D000AFE6C04600100240FFFFFEFFFFFFFBFF28
:1018E000FF1FFFFF00700040FFFEFFFFFFFBFFFF39
:1018F00088130000FFFFFFFEFFE0FFFF2027000826
:10190000000000206D4E6E4A336D80271340336512
:10191000336D6C4ABF0013403365FFF741FB6A4BE0
:101920008146984605E0FFF73BFB4B46C01A404511
:1019300013D8336D3B42F6D107E733683B4333603E
:10194000FFF72EFB804633683B4200D0D3E6FFF71B
:1019500027FB4346C01A6428F5D903204BE7012230
:10196000336893433360FFF71BFB0423070098465B
:1019700004E0FFF715FBC01B0228EED8424633688F
:101980001A42F6D1236857E60122336D934333653B
:10199000FFF706FB02230700984604E0FFF700FB71
:1019A000C01B0228D9D84246336D1A42F6D12368AB
:1019B0008BE63368424A13403360FFF7F1FA802325
:1019C0009B000700984604E0FFF7EAFAC01B0228D4
:1019D000C3D8424633681342F6D1236859E6374DDF
:1019E0003A4A2B68802613402B60FFF7D9FAB604D9
:1019F000070004E0FFF7D4FAC01B0228ADD82B681B
:101A00003342F7D1E16AA36AEA680B4330490A40DE
:101A10001343226B80241343EB6080232A685B040A
:101A200013432B60FFF7BCFA244D0600A40404E026
:101A3000FFF7B6FA801B02288FD82B682342F7D015
:101A40000020D8E61D4A2349936B0B40936380E640
:101A500080231A4ADB0211680B43136013680343A7
:101A6000136022E7154A116D0B4313655AE6012BEB
:101A700000D1BFE6114BA16ADA6880235B021340F4
:101A800001208B4200D0B6E6F023E16A9B031340AD
:101A90008B4200D0AFE6C02000040240206B101A39
:101AA000421E9041C0B2A6E6044B0139186DFF39C1
:101AB00001431965196D0A431A6533E600100240A7
:101AC000FFFEFFFFFFFBFFFF88130000FFFFFFFE8D
:101AD000FFFF02FFFFFFFFEFF8B5CE4647460400C9
:101AE00080B50D0000280DD0012358490A681A401E
:101AF000AA420CD20A689A432A430A600A68134031
:101B0000AB4204D001200CBC90469946F8BD236836
:101B10009A0706D5F0204E49CA688243A06802435E
:101B2000CA60DB0728D54A4A63681268022B52D084
:101B3000032B53D0012B76D09205E3D50321444EDD
:101B4000F2688A431343F360FFF72AFA63680700D9
:101B5000022B58D0032B69D0012B42D00C2398467E
:101B60003C4B994604E0FFF71BFAC01B484548D898
:101B70004246F3681A42F6D10121344A13680B40F9
:101B8000AB4205D913688B43136013681942B9D16E
:101B900023685A0706D52E492F48CA680240E068D4
:101BA0000243CA601B0707D529492369CA682B4825
:101BB000DB0002401343CB60FFF7A6FC244B284A0E
:101BC000DB681B061B0FD35CD840264B1860002037
:101BD000FFF7B2F997E79203B0D493E79201ADD43F
:101BE00090E70B3398461B4B994604E0FFF7D8F972
:101BF000C01B484505D84246F3681340042BF5D175
:101C0000BAE703207FE70A339846124B994604E06F
:101C1000FFF7C6F9C01B4845F3D84246F3681340A6
:101C2000082BF5D1A8E7520788D46BE7093398460B
:101C3000084B994604E0FFF7B3F9C01B4845E0D8CC
:101C40004246F36813400C2BF5D195E70020024083
:101C50000010024088130000FFF8FFFFFFC7FFFFDE
:101C60002027000800000020044B054ADB685B05C4
:101C70005B0FD35C034A1068D840704700100240E5
:101C80003027000800000020044B054ADB689B0455
:101C90005B0FD35C034A1068D840704700100240C5
:101CA0003027000800000020F8B5CE4647460368FC
:101CB00080B504009A062ED580230020604A5B057B
:101CC000916B8046194204D1916B0B4393630123BE
:101CD000984680265B4D76002B6833424DD0656870
:101CE000C020C0212F002A00554E8003336889028E
:101CF00007400A4003409F425FD08A4253D0336D71
:101D0000194000D098E04E490B6D1A4343460A65CE
:101D1000012B42D02368DA0706D503204849CA6C54
:101D20008243A0680243CA649A0706D50C2044493E
:101D3000CA6C8243E0680243CA645A0706D5404928
:101D40004148CA6C024020690243CA641A0706D59A
:101D50003B493E48CA6C024060690243CA640020A5
:101D60001B0606D5364A3A49D36C0B40A1690B4392
:101D7000D3640CBC90469946F8BD2B6833432B6066
:101D8000FFF70EF9070004E0FFF70AF9C01B64280B
:101D900050D82B683342F7D0A1E78B6B2D4A134004
:101DA0008B632368B7E7336801209B03E1D4336D6D
:101DB000134036D0934205D130E0336D194028D01E
:101DC000914226D023689B0623D580211C4E09030F
:101DD000306D376D204B39433165316D1F4F0340F6
:101DE000394031653365C30513D5FFF7D9F8802530
:101DF0001B4B0700AD00994604E0FFF7D1F8C01B6C
:101E0000484517D8336D2B42F7D0C022656892023F
:101E10002A40C0239B029A4200D074E7C027BF0328
:101E20002F40074A0F4913680B401F431760C02219
:101E3000920268E703209CE78A4200D163E7C1E78A
:101E40000010024000700040FFF3FFFFFFCFFFFFD4
:101E5000FFFFF3FFFFFFFFEFFFFFFCFFFFFFF7FFB9
:101E600088130000FFFFCFFF80220368D205904255
:101E700005D00D4A904202D00C4A904207D1702200
:101E800093434A6813430A4A1340CA6813438022A3
:101E900093430A69134303608B68C3620B688362D0
:101EA000012343617047C04600080140001401400F
:101EB000FFFCFFFF70B5041E14D03923C35CDBB2F6
:101EC000002B0AD00223392520686355211DFFF716
:101ED000CBFF01230020635570BD38228354FEF7E9
:101EE0004BFFEFE70120F7E739230222C2540268D3
:101EF000323B91680B40062B03D0012113680B4342
:101F0000136039230122C254002070473923022272
:101F1000C2540368064A196A114203D101211A68A2
:101F20008A431A6039230122C25400207047C046F8
:101F30001111000001210368DA680A43DA60072200
:101F400098680240062A02D01A680A431A600020E4
:101F50007047C04601210368DA688A43DA60186A6C
:101F6000034A104202D11A688A431A60002070475F
:101F700011110000382370B5C25C012A58D0012429
:101F80000222C4540133C25403684B4D9A682A405C
:101F90009A600A68402A00D174E04BD9602A2ED09A
:101FA00057D9702A1BD08024A401A2420FD19A686D
:101FB000424C4D6814408A68C9682A4309020A43A2
:101FC00022439A6080229968D2010A439A60392399
:101FD0000122C2540022013BC254002070BD9A6805
:101FE000364C4D6814408A68C9682A4309020A437E
:101FF000772122439A609A680A439A60E7E710259E
:102000001C6A4A68AC43C9681C629D692C4E09036E
:1020100035402943A0251C6A99617021AC43120107
:1020200022431A629A688A4309390A439A60CEE7C2
:102030000220D3E7102A04D03BD9202A01D0302A2D
:10204000C5D170249968A143693C22430A439A6030
:10205000BDE7502ABBD14D68CA68196A1E6A1201D1
:10206000A6431E62F0269C69B44322430A24A1437E
:1020700029439A61196270219A688A4319390A437F
:102080009A60A4E74D68CA68196A1E6A1201A643DD
:102090001E62F0269C69B44322430A24A1432943CB
:1020A0009A61196270219A688A4329390A439A60B1
:1020B0008DE7002AC5D08AE78800FFFFFF00FFFFF9
:1020C000FF0FFFFF7047C0467047C0467047C046CD
:1020D0007047C0460222036810B5196904000A421D
:1020E00002D0D9680A4254D1042219690A4202D0A6
:1020F000D9680A423AD1082219690A4202D0D9683D
:102100000A4225D1102219690A4202D0D9680A422E
:102110000ED1012219690A4202D0D9680A424ED171
:10212000402219690A4202D0D9680A4241D110BD41
:10213000213A1A6119322276DA69C0239B00200005
:102140001A4243D0FFF7C0FF002323762368E0E75D
:10215000113A1A61DB690D32227620009B0741D0CB
:10216000FFF7B2FF002323762368CBE7093A1A6111
:10217000073222769A69C0239B0020001A422ED192
:10218000FFF7A0FF2000FFF7A1FF002323762368BD
:10219000B1E7053A1A619B69043202769B071BD1AD
:1021A000FFF790FF2000FFF791FF002323762368BD
:1021B0009AE7813A1A612000FFF78AFFB7E7033AEE
:1021C0001A612000FEF794FD2368A9E7FFF77AFF64
:1021D0002000FFF77BFFB7E7FFF776FFE5E7FFF7A4
:1021E00073FFD2E7FFF76EFF2000FFF76FFFB9E73D
:1021F000F0B53825435D012B15D039260223702711
:10220000046883556268A368BA430F6849683A4313
:102210008027BB430B436260A360012383550023E7
:1022200043550020F0BD0220FCE7C046F8B504008D
:102230002569A36802682B436569C1692B4310684F
:10224000804D0B4328400343136053687E4803408E
:10225000E06803437D485360A36982421ED0256A2B
:1022600090682B437A4D284003439360794B9A4200
:1022700000D18CE0784B9A4240D1784BDA6C0C2339
:102280001340774AD35C80221202914244D0082B3B
:1022900000D9D2E0734A9B00D3589F4691686C489E
:1022A00001400B43C021936080226C480901C36C3C
:1022B000D2000B40934200D170E024D98022120159
:1022C000934200D16EE08B4218D180231B026268DA
:1022D00051008918994211D8110399420ED3002751
:1022E0005608190E1802801979410023FDF798FF4E
:1022F0005D4BC2185D4B9A4200D87DE0012000235F
:1023000023666366F8BD002BF8D1FFF7ADFC030030
:102310000020002BDBD1F2E7082BEFD8544A9B00BA
:10232000D3589F46FFF7F0F863685B081818616898
:10233000FDF7EAFE030400201B0C1A004D49103A79
:102340008A42DBD82268D360D9E7FFF79DFC636837
:102350005B081818EBE76368580880231B029C464B
:102360006044E4E7FFF780FC63685B081818DEE769
:102370003A4B61681B684808DB061CD43E4B9C4600
:102380006044FDF7C1FE03041B0C0020D5E7334B6E
:10239000DA6C03231340394AD35C74E7FFF7B4F8CF
:1023A0000300B5E7344A03689446DB063448DB177C
:1023B000034063448BE7334BE1E7FFF7A5F863681D
:1023C00040005B08C0186168FDF79EFE0004000C29
:1023D0000300284A103B934200D98FE70F230200E5
:1023E0009A43130000072268400F1843D060002072
:1023F00085E7FFF749FCE2E72368D86000207EE725
:1024000063686168580880235B029C466044FDF75E
:102410007BFE0004000CDBE7FFF726FCCFE70F4B49
:1024200061681B684808DB060AD5174B9C46604468
:10243000FDF76AFE0004000CCAE7012000237CE7D8
:10244000124BF3E7F369FFEFFFCFFFFF00480040B7
:10245000FFF4FFFF0038014000440040001002403C
:10246000902700084427000800FDFFFFFFFC0F0035
:1024700068270008EFFF00000024F4008C27000804
:1024800000E548FF00093D0000127A000048E8011D
:10249000436A30B5DA0706D50168284C4A682240FD
:1024A000846A22434A609A0706D50168244C4A6828
:1024B0002240C46A22434A605A0706D50168214C6B
:1024C0004A682240046B22434A601A0706D5016815
:1024D0001D4C4A682240446B22434A60DA0606D506
:1024E00001681A4C8A682240846B22438A609A06EB
:1024F00006D50168164C8A682240C46B22438A6064
:102500005A060AD50168134D4A68046C2A402243D2
:102510004A6080225203944209D01B0606D5026805
:102520000D4953680B40816C0B43536030BD4A68C2
:102530000A4C2240446C22434A60EEE7FFFFFDFF55
:10254000FFFFFEFFFFFFFBFFFF7FFFFFFFEFFFFF30
:10255000FFDFFFFFFFFFEFFFFFFFF7FFFFFF9FFF23
:10256000F0B5C64607000C001600984600B5069D5B
:102570003A6801E06B1C0AD1D36923401B1B594206
:102580004B41B342F6D0002004BC9046F0BDFEF7AC
:1025900007FD4346C01AA84201D8002DE8D13B6888
:1025A00008491A6803200A401A609A68A331FF316B
:1025B0008A439A60202300227B67BB675033FA541A
:1025C000E2E7C0465FFEFFFF002330B50400C367AB
:1025D00083B0FEF7E5FC236805001A6812070BD4E8
:1025E0001B685B0717D42023002200206367A367C2
:1025F0005033E25403B030BD80210D4B00220093D4
:10260000890303002000FFF7ABFF00280ED12368E9
:102610001B685B07E7D58021054B00220093C903A7
:102620002B002000FFF79CFF0028DCD00320E1E70F
:10263000FFFFFF0110B5041E27D0436F002B1FD0F2
:102640002423012122686367136820008B431360F1
:10265000FFF7ECFD012818D0636A002B17D123681F
:102660000D495A6820000A402A215A609A688A4314
:102670009A601A6829390A431A60FFF7A5FF10BD4E
:1026800070228354FEF79AFBDAE70120F7E7200077
:10269000FFF7FEFEE3E7C046FFB7FFFF70B5002679
:1026A0000C4D0D4C641BA410A64209D1002600F06D
:1026B0002BF80A4D0A4C641BA410A64205D170BD2C
:1026C000B300EB5898470136EEE7B300EB58984754
:1026D0000136F2E7A8270008A8270008A827000865
:1026E000AC270008002310B59A4200D110BDCC5C85
:1026F000C4540133F8E703001218934200D1704725
:1027000019700133F9E70000F8B5C046F8BC08BC01
:102710009E467047F8B5C046F8BC08BC9E46704758
:102720000000000000000000010203040607080981
:102730000000000001020304030406080C10182026
:1027400030000000642300084A23000870230008BA
:102750003A240008242300083A2400083A240008F8
:102760003A2400085623000818240008F223000821
:102770001E240008FC220008BA230008FC220008DE
:10278000FC220008FC2200080024000801040208C2
:10279000001010100410101002101010080000009B
:0827A000C0DAFF7F0100000018
:0427A800E90000083C
:0427AC00C100000860
:0427B0000000200005
:0400000508000EE5FC
:00000001FF
